BL51 BANKED LINKER/LOCATER V6.00                                                        01/09/2018  11:10:07  PAGE 1


BL51 BANKED LINKER/LOCATER V6.00, INVOKED BY:
C:\KEIL\C51\BIN\BL51.EXE main.obj, Delay_1T.obj TO MA82G5Dxx RAMSIZE (256)


MEMORY MODEL: SMALL


INPUT MODULES INCLUDED:
  main.obj (MAIN)
  Delay_1T.obj (DELAY_1T)
  C:\KEIL\C51\LIB\C51S.LIB (?C_STARTUP)
  C:\KEIL\C51\LIB\C51S.LIB (?C?UIDIV)


LINK MAP OF MODULE:  MA82G5Dxx (MAIN)


            TYPE    BASE      LENGTH    RELOCATION   SEGMENT NAME
            -----------------------------------------------------

            * * * * * * *   D A T A   M E M O R Y   * * * * * * *
            REG     0000H     0008H     ABSOLUTE     "REG BANK 0"
            DATA    0008H     0005H     UNIT         ?DT?MAIN
            IDATA   000DH     0001H     UNIT         ?STACK

            * * * * * * *   C O D E   M E M O R Y   * * * * * * *
            CODE    0000H     0003H     ABSOLUTE     
            CODE    0003H     001FH     UNIT         ?PR?MAIN?MAIN
            CODE    0022H     001BH     UNIT         ?PR?INITIAL_PCA?MAIN
            CODE    003DH     000CH     UNIT         ?C_C51STARTUP
                    0049H     0002H                  *** GAP ***
            CODE    004BH     0003H     ABSOLUTE     
            CODE    004EH     00A9H     UNIT         CODE_DELAY
            CODE    00F7H     0055H     UNIT         ?C?LIB_CODE
            CODE    014CH     001BH     UNIT         ?PR?INITIAL_MCU_SYSCLK?MAIN
            CODE    0167H     0016H     UNIT         ?PR?_PAGEP_WRITE?MAIN
            CODE    017DH     0016H     UNIT         ?PR?_PAGEP_READ?MAIN
            CODE    0193H     0013H     UNIT         ?PR?INT_PCA?MAIN



OVERLAY MAP OF MODULE:   MA82G5Dxx (MAIN)


SEGMENT
  +--> CALLED SEGMENT
---------------------
?C_C51STARTUP
  +--> ?PR?MAIN?MAIN

?PR?MAIN?MAIN
  +--> ?PR?INITIAL_PCA?MAIN
  +--> ?PR?INITIAL_MCU_SYSCLK?MAIN

?PR?INITIAL_MCU_SYSCLK?MAIN
  +--> ?PR?_PAGEP_READ?MAIN
  +--> ?PR?_PAGEP_WRITE?MAIN

BL51 BANKED LINKER/LOCATER V6.00                                                      01/09/2018  11:10:07  PAGE 2




SYMBOL TABLE OF MODULE:  MA82G5Dxx (MAIN)

  VALUE           TYPE          NAME
  ----------------------------------

  -------         MODULE        MAIN
  C:0000H         SYMBOL        _ICE_DUMMY_
  D:0008H         PUBLIC        PCA_Interval
  D:0095H         PUBLIC        P2M0
  D:0092H         PUBLIC        P2M1
  D:0090H         PUBLIC        P1
  D:00A0H         PUBLIC        P2
  D:00E7H         PUBLIC        ISPCR
  D:00C0H         PUBLIC        XICON
  D:00B0H         PUBLIC        P3
  C:0022H         PUBLIC        Initial_PCA
  D:00E8H         PUBLIC        P4
  D:00ADH         PUBLIC        EIE1
  D:00F8H         PUBLIC        P6
  D:00ACH         PUBLIC        SFRPI
  B:00A8H.7       PUBLIC        EA
  D:00F9H         PUBLIC        CH
  C:017DH         PUBLIC        _PageP_Read
  D:00A8H         PUBLIC        IE
  D:00E9H         PUBLIC        CL
  D:00FAH         PUBLIC        CCAP0H
  D:00EAH         PUBLIC        CCAP0L
  D:00DAH         PUBLIC        CCAPM0
  D:00B8H         PUBLIC        IP0L
  C:0167H         PUBLIC        _PageP_Write
  D:00C7H         PUBLIC        CKCON0
  C:0193H         PUBLIC        INT_PCA
  D:00D9H         PUBLIC        CMOD
  D:00D8H         PUBLIC        CCON
  C:0003H         PUBLIC        main
  D:00E6H         PUBLIC        SCMD
  D:00E3H         PUBLIC        IFADRH
  D:00E5H         PUBLIC        IFMT
  D:00E4H         PUBLIC        IFADRL
  D:0088H         PUBLIC        TCON
  D:00E2H         PUBLIC        IFD
  D:000AH         PUBLIC        PCA_Cnt
  D:0098H         PUBLIC        S0CON
  D:000CH         PUBLIC        PCA_Interrupt_Flag
  D:00C8H         PUBLIC        T2CON
  C:014CH         PUBLIC        Initial_MCU_Sysclk
  D:00D0H         PUBLIC        PSW
  -------         PROC          _PAGEP_WRITE
  D:0007H         SYMBOL        Addr
  D:0005H         SYMBOL        Dta
  C:0167H         LINE#         41
  C:0167H         LINE#         42
  C:0167H         LINE#         43
  C:016AH         LINE#         44
  C:016CH         LINE#         45
BL51 BANKED LINKER/LOCATER V6.00                                                      01/09/2018  11:10:07  PAGE 3


  C:016EH         LINE#         46
  C:0171H         LINE#         47
  C:0174H         LINE#         48
  C:0177H         LINE#         49
  C:017AH         LINE#         50
  C:017CH         LINE#         51
  -------         ENDPROC       _PAGEP_WRITE
  -------         PROC          _PAGEP_READ
  D:0007H         SYMBOL        Addr
  -------         DO            
  D:0007H         SYMBOL        Dta
  -------         ENDDO         
  C:017DH         LINE#         53
  C:017DH         LINE#         54
  C:017DH         LINE#         57
  C:0180H         LINE#         58
  C:0182H         LINE#         59
  C:0185H         LINE#         60
  C:0188H         LINE#         61
  C:018BH         LINE#         62
  C:018EH         LINE#         63
  C:0190H         LINE#         65
  C:0192H         LINE#         66
  C:0192H         LINE#         67
  -------         ENDPROC       _PAGEP_READ
  -------         PROC          INT_PCA
  C:0193H         LINE#         69
  C:0193H         LINE#         71
  C:0196H         LINE#         72
  C:0199H         LINE#         73
  C:019CH         LINE#         75
  C:019FH         LINE#         76
  C:01A2H         LINE#         78
  C:01A5H         LINE#         81
  -------         ENDPROC       INT_PCA
  -------         PROC          INITIAL_PCA
  C:0022H         LINE#         83
  C:0022H         LINE#         84
  C:0022H         LINE#         86
  C:0025H         LINE#         87
  C:0028H         LINE#         88
  C:002BH         LINE#         89
  C:002EH         LINE#         90
  C:0030H         LINE#         92
  C:0033H         LINE#         93
  C:0036H         LINE#         94
  C:0039H         LINE#         96
  C:003CH         LINE#         97
  -------         ENDPROC       INITIAL_PCA
  -------         PROC          INITIAL_MCU_SYSCLK
  -------         DO            
  D:0005H         SYMBOL        tmp
  -------         ENDDO         
  C:014CH         LINE#         99
  C:014CH         LINE#         100
  C:014CH         LINE#         105
  C:014FH         LINE#         106
BL51 BANKED LINKER/LOCATER V6.00                                                      01/09/2018  11:10:07  PAGE 4


  C:0156H         LINE#         107
  C:015EH         LINE#         108
  C:0162H         LINE#         109
  -------         ENDPROC       INITIAL_MCU_SYSCLK
  -------         PROC          MAIN
  C:0003H         LINE#         115
  C:0003H         LINE#         116
  C:0003H         LINE#         117
  C:0006H         LINE#         118
  C:0009H         LINE#         119
  C:000BH         LINE#         121
  C:000BH         LINE#         122
  C:000FH         LINE#         123
  C:000FH         LINE#         124
  C:0012H         LINE#         130
  C:0020H         LINE#         132
  C:0020H         LINE#         134
  -------         ENDPROC       MAIN
  -------         ENDMOD        MAIN

  -------         MODULE        DELAY_1T
  C:004EH         SEGMENT       CODE_DELAY
  C:00CFH         PUBLIC        DELAY_100US
  C:00AEH         PUBLIC        DELAY_10US
  C:0091H         PUBLIC        DELAY_1US
  C:00DAH         PUBLIC        DELAY_200US
  C:00B9H         PUBLIC        DELAY_20US
  C:0094H         PUBLIC        DELAY_2US
  C:00EDH         PUBLIC        DELAY_500US
  C:00C4H         PUBLIC        DELAY_50US
  C:004EH         PUBLIC        _DELAY_MS
  D:00E0H         SYMBOL        ACC
  C:00A3H         SYMBOL        DELAY_5US
  C:0079H         SYMBOL        DELAY_UNIT_1MS
  N:0001H         SYMBOL        FOSC_12MHZ
  N:0000H         SYMBOL        FOSC_24MHZ
  C:005CH         SYMBOL        LSB_LOOP
  C:0069H         SYMBOL        MSB_LOOP0
  C:0066H         SYMBOL        MSB_LOOP1
  C:0062H         SYMBOL        NDLSB
  C:0072H         SYMBOL        NDMSB
  C:004EH         LINE#         30
  C:0050H         LINE#         31
  C:0052H         LINE#         32
  C:0054H         LINE#         34
  C:0056H         LINE#         35
  C:0058H         LINE#         37
  C:005AH         LINE#         38
  C:005CH         LINE#         40
  C:005FH         LINE#         41
  C:0062H         LINE#         43
  C:0064H         LINE#         44
  C:0066H         LINE#         46
  C:0069H         LINE#         48
  C:006CH         LINE#         49
  C:006FH         LINE#         50
  C:0072H         LINE#         52
BL51 BANKED LINKER/LOCATER V6.00                                                      01/09/2018  11:10:07  PAGE 5


  C:0074H         LINE#         53
  C:0076H         LINE#         54
  C:0078H         LINE#         55
  C:0079H         LINE#         58
  C:007CH         LINE#         59
  C:007FH         LINE#         60
  C:0082H         LINE#         61
  C:0085H         LINE#         62
  C:0088H         LINE#         63
  C:008BH         LINE#         64
  C:008EH         LINE#         65
  C:008FH         LINE#         66
  C:0090H         LINE#         67
  C:0091H         LINE#         79
  C:0092H         LINE#         79
  C:0093H         LINE#         80
  C:0094H         LINE#         92
  C:0095H         LINE#         92
  C:0096H         LINE#         92
  C:0097H         LINE#         92
  C:0098H         LINE#         92
  C:0099H         LINE#         92
  C:009AH         LINE#         92
  C:009BH         LINE#         92
  C:009CH         LINE#         92
  C:009DH         LINE#         92
  C:009EH         LINE#         92
  C:009FH         LINE#         92
  C:00A0H         LINE#         92
  C:00A1H         LINE#         92
  C:00A2H         LINE#         93
  C:00A3H         LINE#         109
  C:00A5H         LINE#         110
  C:00A8H         LINE#         111
  C:00ABH         LINE#         112
  C:00ADH         LINE#         113
  C:00AEH         LINE#         128
  C:00B0H         LINE#         129
  C:00B3H         LINE#         130
  C:00B6H         LINE#         131
  C:00B8H         LINE#         132
  C:00B9H         LINE#         147
  C:00BBH         LINE#         148
  C:00BEH         LINE#         149
  C:00C1H         LINE#         150
  C:00C3H         LINE#         151
  C:00C4H         LINE#         166
  C:00C6H         LINE#         167
  C:00C9H         LINE#         168
  C:00CCH         LINE#         169
  C:00CEH         LINE#         170
  C:00CFH         LINE#         185
  C:00D1H         LINE#         186
  C:00D4H         LINE#         187
  C:00D7H         LINE#         188
  C:00D9H         LINE#         189
  C:00DAH         LINE#         207
BL51 BANKED LINKER/LOCATER V6.00                                                      01/09/2018  11:10:07  PAGE 6


  C:00DCH         LINE#         208
  C:00DFH         LINE#         209
  C:00E2H         LINE#         210
  C:00E5H         LINE#         211
  C:00E8H         LINE#         212
  C:00EAH         LINE#         213
  C:00EBH         LINE#         213
  C:00ECH         LINE#         214
  C:00EDH         LINE#         235
  C:00F0H         LINE#         236
  C:00F3H         LINE#         237
  C:00F6H         LINE#         238
  -------         ENDMOD        DELAY_1T

  -------         MODULE        ?C?UIDIV
  C:00F7H         PUBLIC        ?C?UIDIV
  -------         ENDMOD        ?C?UIDIV

Program Size: data=14.0 xdata=0 code=420
LINK/LOCATE RUN COMPLETE.  0 WARNING(S),  0 ERROR(S)
